:100000000CC027C026C025C024C023C022C021C0E8
:1000100020C01FC01EC01DC01CC011241FBECFE5C4
:10002000D2E0DEBFCDBF10E0A0E6B0E0E4E2F1E058
:1000300003C0C89531960D92A036B107D1F710E0F4
:10004000A0E6B0E001C01D92A036B107E1F72CD0C8
:1000500068C0D6CF81E088BB87BB12BA82E081BB83
:100060000895262F372F482F592F84E0220F331F52
:10007000441F551F8A95D1F760E079E08DE390E049
:1000800029D02150304029B98AB188618AB90895B0
:100090005F9903C080E090E008958CB1992708959E
:1000A0005D9BFECF8CB9089581E088BB87BB12BAF7
:1000B00082E081BB60E875E280E090E0D2DF5F9B88
:1000C000FECF8CB19927282F8823C9F35D9BFECFE3
:1000D0002CB9F5CFA1E21A2EAA1BBB1BEA2FFB2FCE
:1000E0000DC0AA1FBB1FEE1FFF1FA217B307E40717
:1000F000F50720F0A21BB30BE40BF50B661F771F6F
:10010000881F991F1A9469F760957095809590954E
:10011000262F372F482F592F6A2F7B2F8E2F9F2F57
:040120000895FFCF70
:00000001FF
